:20FFD600E000E000E000E000E000E000E000E000E000E000E000E000E000FD00E000E000EE
:0AFFF600E000E000E000E000E000A1
:20C00000464C094B5420202020005350454349414C50524F472E3F20202000535045432E07
:20C0200050524F47204B4C41523F200050524F4752414D46454C00000000000000414E475A
:20C0400045204B4F443A00000000000000007300204E31202020204E32202020204E332030
:20C0600000492F4F20544553543F00494E47084E4720414B542E3A00555447084E47204189
:20C080004B542E3A0046454C484953544F52494B3F2020202000414E542E50524F472E3AE5
:20C0A000000050554D505449443A0000000044524946545241444552494E472021212000DC
:20C0C00054454D502031204F46465345543A0054454D502032204F46465345543A00736537
:20C0E0006B006D003F002E0050524F4752414D4D4552494E4720202000202000DF43006DF2
:20C10000696E00204D4544202000205554414E200050002000300025006800094E4452413F
:20C12000204B4F443A0000000000000042525954205354520A4D4D454E000000004D415256
:20C140004B45524120494E53502E3F2020005609524D455220534B0A4C4A54414E4B00474D
:20C1600052414E554C4154004449534B415220202000534B0A4C4A45522020005649444151
:20C180005245203D2053544152542020005354094E4720440A5252415220460A520056417A
:20C1A0005454454E46594C4C4E494E4720200046594C4C45522056415454454E2020200081
:20C1C00044524946544B4C4152202020202020200046454C2046594C4C4E494E4720202022
:20C1E000200050524F562050524F4752414D20202020005354094E4720440A525241524EE8
:20C20000412020002020202053544F50504144202020202000202020202020202020202002
:20C2200020202020200046454C2053094B4552482E4E495608200046454C2053094B42526C
:20C24000595441524520200046454C204D4F544F52534B59444420200046454C200A482D5C
:20C26000534B594444202020200046454C2056415454454E545259434B20005354415254BB
:20C280003D4A412020203F3D4E454A004C41444441205354414E444152443F20004C414426
:20C2A0004441205354414E444152443F3F00414E54414C2050524F4752414D3A0000002008
:20C2C0004449534B544944202000000000000000094E445241200A56524947413F202020A2
:20C2E00000534B0A4C4A54454D503A000000000000004449534B54454D503A0000000000F5
:20C3000000000053455041524154494F4E3A000000000000534B0A4C4A5449443A00000094
:20C3200000000000004E495608204449534B3A000000000000004E49560820534B0A4C4A30
:20C340003A000000000000464C094B54205449443A00000000000000534B0A4C4A4D45441A
:20C36000454C000000000000004B4C4152200A565249474120202020200050524F475241F4
:20C380004D4D2E204B4C4152202000454E474C4953483F20202020202020200044455554D0
:20C3A0005343483F2020202020202020004652414E434149533F2020202020202000535651
:20C3C000454E534B413F20202020202020200053554F4D493F2020202020202020202000A0
:20C3E0004E454445524C414E44533F2020202020004954414C49414E4F3F2020202020202E
:20C4000020004E4F52534B3F2020202020202020202000455350414E4F4C3F2020202020FF
:15C420002020200044414E534B3F2020202020202020202000B7
:20C4600046414E202020202020005350454349414C2050524F472E3F202000535045432EC8
:20C4800050524F472E204F4B3F20200050524F4752414D204552524F5200000000494E5054
:20C4A000555420434F44453A0000000000007300204E31202020204E32202020204E33202B
:20C4C00000492F4F20544553543F00494E47084E4720414B542E3A00555447084E47204125
:20C4E0004B542E3A004552524F52204D455353414745532020004E4F2E50524F473A0000B6
:20C50000000050554D5054494D453A00000044524946545241444552494E47202121200029
:20C5200054454D502031204F46465345543A0054454D502032204F46465345543A007365D2
:20C5400063006D003F002E0050524F4752414D4D494E47202020202000202000DF43006DEC
:20C56000696E002057495448200020572F4F202000500020003000250068004348414E47A5
:20C580004520434F44453A00000000005455524E204D414348494E45204F4646004D4152A8
:20C5A0004B20494E5350454354494F4E3F0048454154494E4720424F494C45522020004771
:20C5C00052414E554C4553005741534845532020200052494E53455320202000434F4E54AE
:20C5E000494E5545203D20535441525400434C4F534520444F4F5220464F52202000574156
:20C600005445522D46494C4C494E472020200046494C4C53205741544552202020202000E0
:20C62000524541445920544F2057415348202020004552524F522046494C4C494E47202020
:20C640002000545249414C2050524F4752414D4D452000434C4F534520444F4F52532020F7
:20C6600020202000202020494E544552555054454420202000202020202020202020202036
:20C680002020202020004552524F522053414645204C4556454C004552524F522053414615
:20C6A00045545953572E20004552524F52204D4F544F5250524F5420004552524F522053F3
:20C6C000555045524850524F54004552524F52205741544552505245535300535441525449
:20C6E0003D5945532020203F3D4E4F004C4F4144204445462E56414C5545533F004C4F416B
:20C7000044204445462E56414C5545533F004E4F2E4F462050524F47522E3A000000002017
:20C720005741534854494D4520000000000000004348414E4745204F54482E56414C3F2056
:20C740000052494E53452D54454D503A000000000000574153482D54454D503A00000000EB
:20C7600000000053455041524154494F4E3A00000000000052494E53452D54494D453A0072
:20C7800000000000004C4556454C20574153483A0000000000004C4556454C20424F494CD6
:20C7A00045523A0000000046414E2054494D453A000000000000000052494E534520414721
:20C7C000454E5400000000000046494E4953484544204F54482E56414C0050524F47522E54
:20C7E0002046494E49534845442000454E474C4953483F2020202020202020004445555434
:20C800005343483F2020202020202020004652414E434149533F20202020202020005356EC
:20C82000454E534B413F20202020202020200053554F4D493F20202020202020202020003B
:20C840004E454445524C414E44533F2020202020004954414C49414E4F3F202020202020C9
:20C8600020004E4F52534B3F2020202020202020202000455350414E4F4C3F20202020209B
:15C880002020200044414E534B3F202020202020202020200053
:20C8C0004C0E46544552202020005350455A49414C2050524F472E3F2020005350455A2EE0
:20C8E00050524F472E204F4B3F20200050524F4752414D4D204645484C45520000434F4488
:20C90000452045494E474542454E3A0000007300204E31202020204E32202020204E332008
:20C9200000492F4F20544553543F00494E47084E4720414B542E3A00555447084E472041C0
:20C940004B542E3A004645484C45524D454C44554E47454E2000414E5A2E50524F472E3AA4
:20C96000000050554D504544415545523A0044524946545241444552494E4720212120003E
:20C9800054454D502031204F46465345543A0054454D502032204F46465345543A0073656E
:20C9A0006B006D003F002E0050524F4752414D4D494552554E47202000202000DF43004D14
:20C9C000696E00204D4954202000204F484E452000500020003000250068004E4555455220
:20C9E00020434F44453A0000000000005354524F4D2041425354454C4C454E0000494E5389
:20CA0000502E204D41524B4945522E3F2000484549545A5420424F494C4552202020004784
:20CA200052414E554C41540053500E4C454E202020004B4C415253500E4C2000574549546F
:20CA40004552203D205354415254202000540E5245205343484C49455353454E2000460E76
:20CA60005220574153534552460E4C4C454E00460E4C4C542057415353455220202020003B
:20CA800042455452494542534245524549542020004645484C455220460E4C4C454E2020B6
:20CAA0002000564552535543482050524F4752414D4D00540E5245205343484C494553533A
:20CAC000454E20002050524F4752414D4D53544F50502020002020202020202020202020E8
:20CAE0002020202020004645484C2E534943482E4E4956454155004645484C2E53494348B8
:20CB00002E534348414C54004645484C2E204D4F544F525343482E20004645484C200E4869
:20CB20002D53434855545A2020004645484C2E574153534552445255434B0053544152547E
:20CB40003D4A4120203F3D4E45494E005745524B5357455254204C4144454E3F00574552A8
:20CB60004B5357455254204C4144454E3F00414E5A2E2050524F4752414D4D3A000000201C
:20CB800053500E4C5A4549542000000000000000414E442E574552544520094E44524E3F1A
:20CBA000004B4C415253500E4C544D503A000000000053500E4C54454D503A0000000000B6
:20CBC00000000041425452454E4E44415545523A000000004B4C415253500E4C444155524D
:20CBE0003A000000004E49562E2053500E4C454E3A00000000004E49562E20424F494C4550
:20CC0000523A00000000004C0E4654455244415545523A00000000004B4C415253502E4D0A
:20CC200049544C000000000000414E44455245205745525445204F4B3F0050524F475241F1
:20CC40004D2E204645525449473F00454E474C4953483F20202020202020200044455554BE
:20CC60005343483F2020202020202020004652414E434149533F2020202020202000535688
:20CC8000454E534B413F20202020202020200053554F4D493F2020202020202020202000D7
:20CCA0004E454445524C414E4453202020202020004954414C49414E4F3F20202020202084
:20CCC00020004E4F52534B3F2020202020202020202000455350414E4F4C3F202020202037
:15CCE0002020200044414E534B3F2020202020202020202000EF
:20CD200056454E54494C4552200050524F472E205350454349414C453F200050524F472ED9
:20CD400020535045432E204F4B3F200050524F4752414D4D452045525245555200494E53B8
:20CD60004552455220434F44453A000000007300204E31202020204E32202020204E3320DD
:20CD800000492F4F20544553543F00494E47084E4720414B542E3A00555447084E4720415C
:20CDA0004B542E3A00414646495343482E2045525245555220004E425245205047522E3A9D
:20CDC00000004455520B4520504D503A000044524946545241444552494E4720212120008A
:20CDE00054454D502031204F46465345543A0054454D502032204F46465345543A0073650A
:20CE000063006D003F002E0050524F4752414D4D4154494F4E20202000202000DF43006DC6
:20CE2000696E00204156454320002053414E532000500020003000250068004E4F5556458D
:20CE4000415520434F44453A00000000455441494E445245204D4143482E000000504F492C
:20CE60004E54204420494E53504543542E004D495345200D2054454D5020424F552E00471C
:20CE800052414E554C4553004C41564520202020200052494E43452020202000434F4E548B
:20CEA000494E5545203D205354415254004645524D455420504F525445532050520052451D
:20CEC0004D504C49535341474520454155200052454D504C495420454155202020202000DA
:20CEE00050520C5445204155204C415641474520004552524555522052454D504C495353E1
:20CF00002E005047522E204558504552494D454E5420004645524D455420504F52544553CB
:20CF20002020200020202020204152520C542020202020200020202020202020202020208C
:20CF40002020202020004552522E4E4956454155205345435552004552522E494E54455217
:20CF600052205345435552004552522E5345435552204D4F54455552004552522E20534559
:20CF800055522053555243482E004552522E2050524553532045415520200053544152548A
:20CFA0003D4F554920203F3D4E4F4E0056414C2E4445462E205553494E453F200056414CAC
:20CFC0002E4445462E205553494E453F3F004E4252452044452050524F47522E3A00002002
:20CFE0004455522E4C41562E20000000000000004348414E474520415554522056414C3FA3
:20D0000000544D502052494E0F4147453A000000000054454D50204C41564147453A0000C0
:20D020000000004455522E20534550415241543A000000004455522E2052494E0F4147456F
:20D040003A000000004E49562E204C41564147453A00000000004E49562E20424F55494CBB
:20D060004C3A00000000004455522E56454E54494C2E3A00000000004147454E54205249AD
:20D080004E0F2E00000000000050520C54204155545245533F202020200050524F47522E98
:20D0A0005445524D494E0B453F2000454E474C4953483F2020202020202020004445555477
:20D0C0005343483F2020202020202020004652414E434149533F2020202020202000535624
:20D0E000454E534B413F20202020202020200053554F4D493F202020202020202020200073
:20D100004E454445524C414E44533F2020202020004954414C49414E4F3F20202020202000
:20D1200020004E4F52534B3F2020202020202020202000455350414E4F4C3F2020202020D2
:15D140002020200044414E534B3F20202020202020202020008A
:20D18000505548414C4C494E20004552494B4F49534F484A2E3F20202020004F484A454CBC
:20D1A0004D4F494E5449204F4B3F20004F484A454C4D4156495248452000000000414E4E0B
:20D1C00041204B4F4F44493A0000000000007300204E31202020204E32202020204E33200B
:20D1E00000492F4F20544553543F00494E47084E4720414B542E3A00555447084E472041F8
:20D200004B542E3A0056494B41484953544F52494120202020004F484A454C2E4C4B4D3A3B
:20D22000000050554D50505541494B3A000044524946545241444552494E472021212000B1
:20D2400054454D502031204F46465345543A0054454D502032204F46465345543A007365A5
:20D260006B006D003F002E004F484A454C4D4F494E5449202020202000202000DF43004DD8
:20D28000494E00202B2020202000202D2020202000500020003000250068005641494844C6
:20D2A00041204B4F4F44493A000000004B41544B414953452056495254413A00004B49524A
:20D2C0004A41205441524B49535455533F0048555548542E564544454E204C094D4D00520B
:20D2E0004145504553552000504553552020202020004855554854454C5520004A41544BB0
:20D3000041203D2053544152542020200053554C4A45204F56455420202020202000564525
:20D3200044454E54095954540A202020202000540959540909205645545409202020200006
:20D340004B095954540A56414C4D4953202020200056090952092054095954540A20202077
:20D3600020004B4F454F484A454C4D412020202020200053554C4A45204F564554202020AD
:20D38000202020005649524845205059530959544554545900202020202020202020202037
:20D3A000202020202000564952484520545552564152414A412000564952484520545552C6
:20D3C00056414B59544B2E005649524845204D4F4F54544F524920200056495248452059F3
:20D3E0004C494B55554D2E202000564952484520564553495041494E4520005354415254F8
:20D400003D202B2020203F3D202D20004C415441412056414B494F3F20202020004C41549E
:20D4200041412056414B494F3F3F202020004F484A454C4D49454E204C4B4D3A00000020F9
:20D440005045535541492E3A20000000000000004D55555441204D555554203F20202020A7
:20D460000048555548542E4C094D503A000000000000504553554C094D500A543A000000FD
:20D4800000000052454B45455420504F4C533A000000000048555548542E41494B413A0028
:20D4A0000000000000414E5455524920504553553A0000000000414E54555249204855551D
:20D4C00048543A00000000505548414C4C2E41494B413A000000000048555548542E4149EC
:20D4E0004E453A0000000000004D5555542056414C4D49533F20202020004F484A454C4DAA
:20D50000412056414C4D49533F2000454E474C4953483F2020202020202020004445555404
:20D520005343483F2020202020202020004652414E434149533F20202020202020005356BF
:20D54000454E534B413F20202020202020200053554F4D493F20202020202020202020000E
:20D560004E454445524C414E44533F2020202020004954414C49414E4F3F2020202020209C
:20D5800020004E4F52534B3F2020202020202020202000455350414E4F4C3F20202020206E
:15D5A0002020200044414E534B3F202020202020202020200026
:20D5E00056454E54494C41542000535045432E50524F472E5354414E443F00535045432ED3
:20D600002050524F472E204F4B3F200050524F4752414D4D4120464F55540000005741438C
:20D620004854574F4F52443A0000000000007300204E31202020204E32202020204E332056
:20D6400000492F4F20544553543F00494E47084E4720414B542E3A00555447084E47204193
:20D660004B542E3A00464F5554204D454C44494E47454E20200041414E542E50524F473AAE
:20D680000000504F4D5054494A443A00000044524946545241444552494E472021212000A2
:20D6A00054454D502031204F46465345543A0054454D502032204F46465345543A00736541
:20D6C00063006D003F002E0050524F4752414D4D4552454E2020202000202000DF43004D4F
:20D6E000494E00204D4554202000204745454E2000500020003000250068004E4945555739
:20D700002E5741434854573A00000000484F4F4644534348414B2E2055495400004E415AD0
:20D72000494348542050554E543F20202000564552572E20424F494C455220202020004BA1
:20D740004F5252454C53200057415353454E202020004E4153504F454C202000564552441E
:20D760004552203D20535441525420200044554552454E20534C554954454E202000564FDB
:20D780004F522056554C4C454E20202020200056554C5420574154455220202020202000A4
:20D7A0004B4C415220562E2057415353454E202000464F55542056554C2020202020202035
:20D7C0002000544553542050524F4752414D4D41202000534C5549542044455552454E204F
:20D7E0002020200050524F47522E4F4E44455242524F4B2E002020202020202020202020DD
:20D80000202020202000464F55542057415445524E495645415500464F5554204445555231
:20D82000534348414B202000504F4D50204F56455242454C415354200044524F4F474B4FB6
:20D840004F4B20424556202020004C4147452057415445524452554B202000535441525411
:20D860003D4A412020203F3D4E454500464142522E494E5354454C4C2E3F20200046414252
:20D88000522E494E5354454C4C2E3F3F200041414E542E50524F4752414D2E3A000000202F
:20D8A00057415354494A443A2000000000000000414E44455245204745472E57494A5A3FA5
:20D8C000004E4153504F4C54454D503A00000000000057415354454D503A000000000000B0
:20D8E0000000004E412057415353454E3A000000000000004E4153504F4C54494A443A003C
:20D9000000000000004E49562E2057415354414E4B3A000000004E49562E20424F494C45D3
:20D92000523A000000000056454E542E2054494A443A0000000000004E4153504F454C4D0C
:20D9400049442E000000000000414E44455245204745472E204F4B3F200050524F47524158
:20D960004D2E4B4C4141523F202000454E474C4953483F20202020202020200044455554C7
:20D980005343483F2020202020202020004652414E434149533F202020202020200053565B
:20D9A000454E534B413F20202020202020200053554F4D493F2020202020202020202000AA
:20D9C0004E454445524C414E44533F2020202020004954414C49414E4F3F20202020202038
:20D9E00020004E4F52534B3F2020202020202020202000455350414E4F4C3F20202020200A
:15DA00002020200044414E534B3F2020202020202020202000C1
:20DA800056454E544F4C4120200050524F47522E205350454349414C453F0046494E45208E
:20DAA00050524F472E535045432E3F004552524F52452050524F4752414D4D4100434F44FD
:20DAC00049434520494E5055543A000000007300204E31202020204E32202020204E332058
:20DAE00000492F4F20544553543F00494E47084E4720414B542E3A00555447084E472041EF
:20DB00004B542E3A004552524F524520202020202020202020004E522E505247523A0000AC
:20DB200000004F524520504F4D50413A000044524946545241444552494E472021212000E1
:20DB400054454D502031204F46465345543A0054454D502032204F46465345543A0073659C
:20DB600063006D003F002E0050524F4752414D4D415A494F4E45202000202000DF43004D4E
:20DB8000494E0020434F4E2020002053454E5320005000200030002500680043414D4249AC
:20DBA0004120434F442E3A0000000000535045474E49204D41434348494E410000535049C0
:20DBC0004120434F4E54524F4C4C4F3F200052495343414C444920424F494C45522000473A
:20DBE00052414E554C4920004C41564120202020200053434941435155412000434F4E54D8
:20DC0000494E554F203D2053544152540043484955444920504F52544520504552005249BC
:20DC2000454D50494D2E2041435155412020005249454D504945204143515541202020007D
:20DC40004F4B204C4156414747494F2020202020004552524F5245204C4956454C4C4F20FA
:20DC6000200050524F4752414D4D412050524F56412000434849555355524120504F52544D
:20DC800045202000202020204152524553544F20202020200020202020202020202020205F
:20DCA0002020202020004552522E204C49562E2053494355522E004552522E204D4943523E
:20DCC0004F20504F525441004552522E2050524F54455A2E4D4F542E004552522E20535509
:20DCE0005252495343414C442E004552522E2050524553532E4143515541005354415254B7
:20DD00003D5349202020203F3D4E4F0050524F4752414D4120424153453F20200050524F8D
:20DD20004752414D4120424153453F3F20004E522E2050524F4752414D4D493A00000020AC
:20DD40004455522E4C41563A20000000000000005641522E20414C5452492056414C3F2058
:20DD60000054DF20534349414351554F3A000000000054DF204C4156414747494F3A0000E7
:20DD80000000004455522E205345504152415A3A000000004455522E534349414351554F89
:20DDA0003A000000004C49562E4C4156414747494F3A000000004C49562E20424F494C45E8
:20DDC000523A00000000004455522E56454E54494C2E3A00000000004252494C4C49414E17
:20DDE000542020000000000000414C54524920564F4C4F5249204F4B3F0046494E4520508D
:20DE0000524F4752414D4D413F2000454E474C4953483F20202020202020200044455554D2
:20DE20005343483F2020202020202020004652414E434149533F20202020202020005356B6
:20DE4000454E534B413F20202020202020200053554F4D493F202020202020202020200005
:20DE60004E454445524C414E44533F2020202020004954414C49414E4F3F20202020202093
:20DE800020004E4F52534B3F2020202020202020202000455350414E4F4C3F202020202065
:15DEA0002020200044414E534B3F20202020202020202020001D
:20800000564946544520202020005350455349414C50524F472E3F20202000535045432EF3
:2080200050524F472E4B4C41523F200050524F4752414D4645494C2020202020004B4F449B
:20804000453A0000000000000000000000007300204E31202020204E32202020204E33206E
:2080600000492F4F20544553543F00494E47084E4720414B542E3A00555447084E472041C9
:208080004B542E3A004645494C484953544F52494B20202020004E522E505247523A000089
:2080A000000050554D50455449443A00000044524946545241444552494E472021212000D7
:2080C00054454D502031204F46465345543A0054454D502032204F46465345543A00736577
:2080E0006B006D003F002E0050524F4752414D4D4552494E4720202000202000DF43006D32
:20810000696E00204D4544202000205554454E200050002000300025006800454E4452453B
:20812000204B4F44453A0000000000004252595420535452304D4D454E000000004D455227
:208140004B20494E53502E3F2020202020005641524D455220534B594C4C54414E4B00477C
:2081600052414E554C4154005641534B455220202000534B594C4C4552202000564944452E
:208180005245203D2053544152542020005354454E4720444F52454E4520464F5200564101
:2081A0004E4E46594C4C4E494E47202020200046594C4C45522056414E4E2020202020007F
:2081C0004452494654534B4C4152202020202020004645494C204D45442046594C4C494EE5
:2081E00047005445535450524F4752414D2020202020005354454E4720444F52454E4520C2
:20820000202020002020202053544F5050455420202020200020202020202020202020204F
:208220002020202020004645494C2053494B4B45482E4E49562E004645494C2053494B4BE4
:208240002E425259542E20004645494C204D4F544F525645524E2020004645494C20542E53
:208260004B2E53494B522E2020004645494C2056414E4E545259434B202000535441525410
:208280003D4A412020203F3D4E4549005354442E20564552444945523F202020005354448A
:2082A0002E20564552444945523F3F202000414E54414C4C2050524F4752414D3A00002053
:2082C0005641534B5449443A2000000000000000454E44524520414E4E45543F202020206B
:2082E00000534B594C4C4554454D503A2000000000005641534B4554454D503A20200000F0
:20830000000000534550455241534A4F4E3A000000000000534B594C4C455449443A00003A
:2083200000000000004E495641205641534B3A000000000000004E49564120534B594C4CA3
:208340003A00000000000056494654455449443A0000000000000000544F5252454D4944E4
:2083600044454C0000000000004F2E4B2E20414E4E45543F20202020200050524F475241F2
:208380004D204F2E4B2E3F20202000454E474C4953483F2020202020202020004445555460
:2083A0005343483F2020202020202020004652414E434149533F2020202020202000535691
:2083C000454E534B413F20202020202020200053554F4D493F2020202020202020202000E0
:2083E0004E454445524C414E44533F2020202020004954414C49414E4F3F2020202020206E
:2084000020004E4F52534B3F2020202020202020202000455350414E4F4C3F20202020203F
:158420002020200044414E534B3F2020202020202020202000F7
:2084600056454E54494C4152200050524F472E2045535045432E3F2020200050524F472E4E
:208480002045535045432E204F4B3F004552524F522050524F4752414D41202000494E54F7
:2084A000524F20434F4449474F3A000000007300204E31202020204E32202020204E3320D9
:2084C00000492F4F20544553543F00494E47084E4720414B542E3A00555447084E47204165
:2084E0004B542E3A004D454E53414A4553204552524F522020004E522E505247523A0000F2
:2085000000004455522E424F4D42413A000044524946545241444552494E47202121200060
:2085200054454D502031204F46465345543A0054454D502032204F46465345543A00736512
:2085400063006D003F002E0050524F4752414D4D4143494F4E20202000202000DF43006DE0
:20856000696E0020434F4E2020002053494E2020005000200030002500680043414D424911
:208580004520434F442E3A0000000000415041474152204D415155494E410000004D415280
:2085A00043415220494E53504543432E3F0043414C454E54414E444F20424F494C5200479B
:2085C00052414E554C4F20004C4156414E444F20200041434C415241444F2000434F4E54DA
:2085E000494E5541523D205354415254004345525241522050554552544120202000504170
:208600005241204C4C454E4152204147554100434F4749454E444F204147554120202000C5
:208620005055454445204C415641522020202020004552524F52204C4C454E41444F2020A8
:20864000200050524F4752414D4120444520544553540043455252415220505545525441E8
:20866000202020002020494E544552555043494F4E2020200020202020202020202020204A
:208680002020202020004552522E4E4956454C2053454755522E004552522E53454E532E53
:2086A00020505545525441004552522E204D4F544F522D50524F542E004552522E50524F59
:2086C0005445432E5445524D2E004552522E50524553494F4E204147554100535441525427
:2086E0003D53492020203F3D4E4F4E00204441544F5320464142524943413F200020444133
:20870000544F5320464142524943413F3F004E522E2050524F4752414D413A00000000203C
:208720004455522E4C41563A200000000000000020434F4D422E4F54524F532056414C3F9B
:208740000054DF2041434C415241444F3A000000000054DF204C415641444F3A0000000011
:2087600000000053455041524143494F4E3A0000000000004455522E41434C415241444F8A
:208780003A000000004E49562E2054414E5155453A00000000004E49562E20424F494C45B6
:2087A000523A00000000004455522E56454E54494C2E3A000000000050524F442E204252C3
:2087C000494C4C4F0000000000204F54524F2056414C2E204F4B3F2020002046494E414C11
:2087E0002050524F4752414D413F00454E474C4953483F2020202020202020004445555446
:208800005343483F2020202020202020004652414E434149533F202020202020200053562C
:20882000454E534B413F20202020202020200053554F4D493F20202020202020202020007B
:208840004E454445524C414E44533F2020202020004954414C49414E4F3F20202020202009
:2088600020004E4F52534B3F2020202020202020202000455350414E4F4C3F2020202020DB
:158880002020200044414E534B3F202020202020202020200093
:2088C00056454E54494C415420005350454349414C50524F472E3F20202000535045432EB2
:2088E00050524F47204B4C41523F200050524F4752414D46454A4C2020202020004B4F44E0
:20890000453A0000000000000000000000007300204E31202020204E32202020204E3320A5
:2089200000492F4F20544553543F00494E47084E4720414B542E3A00555447084E47204100
:208940004B542E3A0046454A4C484953544F52494B3F20202000414E542E50524F472E3A32
:20896000000050554D50455449443A00000044524946545241444552494E4720212120000E
:2089800054454D502031204F46465345543A0054454D502032204F46465345543A007365AE
:2089A0006B006D003F002E0050524F4752414D4D4552494E4720202000202000DF43006D69
:2089C000696E00204D4544202000205544454E20005000200030002500680041454E445287
:2089E00045204B4F44453A0000000000534C554B20535452304D4D454E000000004D415220
:208A00004B455220494E53502E3F202020005641524D455220534B594C4C54414E4B00475C
:208A200052414E554C4154005641534B455220202000534B594C4C45522020005649444565
:208A40005245203D2053544152542020004C554B20443052454E4520464F522020005641AC
:208A60004E44500846594C444E494E47202000500846594C4445522056414E4E20202000A0
:208A800044524946544B4C4152202020202020200046454A4C204D2E2046594C444E494E63
:208AA00047005445535450524F4752414D2020202020004C554B20443052454E452020206D
:208AC000202020002020202053544F50504554202020202000202020202020202020202087
:208AE00020202020200046454A4C2053494B4B4552482E4E49560046454A4C20444F524BF8
:208B00004F4E54414B54200046454A4C204D4F544F52564145524E200046454A4C20542E33
:208B20004B2E53494B522E20200046454A4C2056414E445452594B20202000535441525473
:208B40003D4A412020203F3D4E454A005354442E20564552444945523F20202000535444C0
:208B60002E20564552444945523F3F202000414E54414C2050524F4752414D3A00000020D6
:208B80005641534B4554443A200000000000000041454E445245204F56524947413F202053
:208BA00000534B594C4C4554454D503A0000000000005641534B4554454D503A0000000087
:208BC00000000053455041524154494F4E3A000000000000534B594C4C455449443A000076
:208BE00000000000004E4956454155205641534B3A00000000004E495645415520534B593F
:208C00004C3A000000000056454E54494C2E5449443A000000000000544F5252454D49444D
:208C200044454C0000000000004B4C4152204F56524947453F202020200050524F475241BF
:208C40004D204F2E4B2E3F20202000454E474C4953483F2020202020202020004445555497
:208C60005343483F2020202020202020004652414E434149533F20202020202020005356C8
:208C8000454E534B413F20202020202020200053554F4D493F202020202020202020200017
:208CA0004E454445524C414E44533F2020202020004954414C49414E4F3F202020202020A5
:208CC00020004E4F52534B3F2020202020202020202000455350414E4F4C3F202020202077
:158CE0002020200044414E534B3F20202020202020202020002F
:20B0000018CE6002BD94C0BD94C018CE6002181D00A0181C00408630BD93678630BD93675B
:20B020008630BD93678620BD93678628BD9424BD94C08606BD9424BD94C08614BD9424BD34
:1BB0400094C0860CBD9424BD94C08601BD9424BD94C018CE6002181C002039A7
:20FF000001010A141E28323C46505152535455565758595AFF01010A141E28323C3D3E3F93
:20FF200040414243444546FF0A141E28323C000A0F14191E23282D32373C00000000010396
:14FF400000010600000300000000FF00010F1E2D3C4B5AFF69
:20FD0000DD66DF6818DF6A132902107F0035BDEB852608BDEB8B26031529021329400B7CFC
:20FD200000539653810F2E0D20177A0053965381002702200C13294005152940200314299A
:20FD4000401329010EBDEB027C0065966581072E07200B7F00652006BDEB7E152901132800
:20FD600020037C0036132840037C0037132810037C00357C003C860A913C2E33132680054A
:20FD8000DE3008DF307C00521427107C00327C00347C003F7C004013288007DC38C30001B6
:20FDA000DD387C00337F003C132802037C0051963D27087A003D2603152704963E27087A18
:14FDC000003E26031527088640B71025DC66DE6818DE6A3BAF
:20E000008600B710248693B710397F10358683B71026863EB710098E00FF8600B760018677
:20E02000FFB760008604B760018600B7600386E0B760028604B76003BD938618CE01F4BDF7
:20E040009323BDF706861497B77F000B7F001E7F001FBDF7F0BDF154BDF706BDF8A5BDE943
:20E06000DEBDE9B0BDED39B6103181FF27037EE084BDED6BB6103281FF27037EE084BDF7B9
:20E08000067EA13886009700BD9452BDEB972700BDEB8B27061527407EA0007EE2801527E7
:20E0A00041BD9452CCC096BDEEB3DC18BDEDBABD9474CCC0A2BDEEB3DC1ABDEDBACCC11953
:20E0C000BDEEB3BD9623122501F9BD9452B6B7159764B6B71497639705CCC0C0BDF0029772
:20E0E00063CEB714BD95F096649705CCC0CFBDF0029764CEB715BD95F018CE01F4BD93231D
:20E10000BD9452BD9474CCC050BDEEB38681BD9496BDEC199604BDED9DCCC113BDEEB38648
:20E1200087BD9496BDEC519604BDED9DCCC113BDEEB3868DBD9496BDEC899604BDED9DCCBF
:20E14000C113BDEEB3BDE688962A27037EE5D2BDEB8B262120B6BD9452CCC061BDEEB3BD48
:20E160009474CCC27BBDEEB3BD9623122501067E921B7EE24D142901BD947ACCC085BDEEDF
:20E18000B3BD9474CCC27BBDEEB3BD9623122501E1BD947ACCC215BDEEB3BD947ACEB7E015
:20E1A000A600BDED9DCCC0E6BDEEB3CEB7E0A601BDED9DCCC0E6BDEEB3CEB7E0A602BDEDC8
:20E1C0009DCCC0E6BDEEB3CEB7E0A603BDED9DCCC0E6BDEEB3CEB7E0A604BDED9DBD9623E1
:20E1E000BD947ACCC215BDEEB3BD947ACEB7E0A605BDED9DCCC0E6BDEEB3CEB7E0A606BD93
:20E20000ED9DCCC0E6BDEEB3CEB7E0A607BDED9DCCC0E6BDEEB3CEB7E0A608BDED9DCCC095
:20E22000E6BDEEB3CEB7E0A609BDED9DBD9623BD947ACCC215BDEEB3BD947ACCC13DBDEEBD
:20E24000B3BD9623122501058663BDF22DBD9452CCC1E2BDEEB3BD9474CCC27BBDEEB3BD3A
:20E2600096231225010486019700BD947ACCC01BBDEEB3BD9623122501037EF4817EE09E1B
:20E28000152902BDF8A5142740BDF706BD9452960C972B960D972C7F0030142680BDEB171A
:20E2A000CC00051A93302EF8BDEB17152680152703152701BDE921962A27037EE5D2BDEC05
:20E2C000192646152730BD947ACCC18DBDEEB3BD9474CCC19EBDEEB3BD9623122501F9BD58
:20E2E000E97F8602912A27D68601912A27C3142730BD9452BD9474CCC1AFBDEEB314273270
:20E30000BDE8568601912A27A81427038601971E142730BDE9217F0030142904142680BDDE
:20E320009474CCC1C0BDEEB3BD9623122501F9152904BDE921962A27037EE66015298014FA
:20E340002730BD9474CCC215BDEEB3BD9474CCC111BDEEB3961E961EBDED9DCCC113BDEEE5
:20E36000B3BDE6149654BDED9DCCC0FFBDEEB3CCC113BDEEB3962D81002706CCC15FBDEE13
:20E38000B3CC0000DD30142908142680BD96231225020F7C001E960E911E2CA08601971E3F
:20E3A000209A1529081526802000BD9474CCC215BDEEB3142730142980BDE6147F00307FAF
:20E3C0000031142680BDE688962A27037EE5D2CC00031A93302EEEBDE97F962A27037EE5CE
:20E3E000D218CE07D0BD9334BDE856962A27037EE33CCC0000DD30BDEAD8BDEAEDBDE68871
:20E40000962A27037EE5D2BDEEF8CC000B1A93302EEBBDEAD1BDE688962A27037EE5D2BDEE
:20E42000EEF8CC00161A93302EEBBDEACACCC168DD55142780BDE688962A27037EE5D2BDC4
:20E44000EEF8CC001B1A93302EEB4F912D2703BDEAE6BDE688962A27037EE5D2BDEEF8CC7C
:20E46000001BD32E1A93302EE9BDEB48BDE688962A27037EE5D2BDEEF8CC001BD32ED36193
:20E480001A93302EE7152680BDEB2C18CE01F4BD9323BDEB3318CE01F4BD9323BDEB3A188A
:20E4A000CE01F4BD9323BDEB4F18CE01F4BD9323BDECFD2615BD9474CCC215BDEEB31527FE
:20E4C00080BD9474CCC14EBDEEB3BDE688962A27037EE5D27A002C7A002CBDECFD27022039
:20E4E000087C002C7C002C20E17C002C7C002CBDEADF18CE01F4BD9323BDEAF4142680CC7E
:20E50000C172DD55142780BDE688962A27037EE5D2DC5FC3001BD32ED3611A93302EE8BD93
:20E52000EB41BD938618CE01F4BD9323BDEB63DC121A8300002725CCC000DD55BDEABCBDCB
:20E54000E688962A27037EE5D2DC5FC30028D32ED361D3121A93302EE6BDEB1E960081011F
:20E560002727152680152780BD9474CCC215BDEEB3BD93867F00307F0031142730152980B2
:20E58000BDEF85BDE9217EE33CBDEF851527B0BD9474CCC215BDEEB3BD9386BD9452BDE9E4
:20E5A00021CCC168DD55CCC1E2BDEEB31426807F00307F0031BDE688962A27037EE5D2BD26
:20E5C000EB8B2608CC02321A93302EE9BD94527EE3AA8601912A26037EE2B18602912A2610
:20E5E000037EE2BE8607912A26037EE33C860A912A26037EE280860B912A26037EF2EB8642
:20E600000C912A26037EE09E860D912A26037EF0397EEA9B961EC6033DC3007B8FA6009729
:20E620002D08A60097549704C6B73DDD2E9610C6033DDD61D32EDD57960FC6033DDD5FD3DB
:20E6400057DD579611498102270BC6033DDD12D357DD572005CC000020F3C30028DD5739DB
:20E66000BDE9B0BD947ABD9474CCC204BDEEB318CE01F4BD9323BD9474CCC215BDEEB31898
:20E68000CE01F4BD932320DBBD947ABDEE58132904037EF275132908037EF29113272007AA
:20E6A00013271003BDEDCD13270128BDEC892623860F913F2E20BD947A152730CCC226DD3D
:20E6C00046BDEEB38605BDF22D152701BDEA39BDE660397F003FBDEBA32657BDEB9D265293
:20E6E000BDEB8B274212280149142810860A91352E46BDE9DEBDE9B0142801BDE9B015273B
:20E7000080BDEBA3260315270C142730BD9452BDE921152801132701058607972A3986015C
:20E72000972A39270920B9BDEB85270620B7270220AE1528107F00357A002BBDEC89271D92
:20E74000BDECC12618BDEC0D26137C002B7A002B7A002BBDECC1260DBDEAA720087C002B77
:20E76000BDEB0920067C002B7C002B7A002CBDEC512722BDECFD261D7C002C7A002C7A00DA
:20E780002CBDECFD2617BDEBFB2612BDEC13260DBDEAAE20087C002CBDEB1020067C002CF5
:20E7A0007C002CBDEBB6271B1228081E142808BD9452CCC248DD46BDEEB38608BDF22DBD4C
:20E7C000EA3939BDEBC3270220DEBDEBE32720BDEBA9271B12280423142804BD9452CCC214
:20E7E00059DD46BDEEB38609BDF22DBDEA3939BDEBE92707BDEBD0270220D913270217BD52
:20E80000EC132612BDEC51260D142880CC044C1A93382E11201A1528807F00381228022787
:20E82000BDEB25202DBDEAC37F00511428022022BDEB25BD9452CCC26ADD46BDEEB3860A8B
:20E84000BDF22DBDEA3939860691512E0515280220CE7F002A397F003ABDE688962A270147
:20E8600039BDEC892709BDEC1927047F002A39BDECC1261B7A002C7A002CBDECFD27087CE6
:20E88000002C7C002C20087C002C7C002C20CABDEC5127C5BDE688962A270139122802F4E0
:20E8A0007F003418CE03E8BD9323BDEADF96142703BDEAF4BDE688962A2701399634815B7A
:20E8C0002E1BBDEC1927ED7F0052BDE688962A270139BDEC1927DD861991522EEDBDEB41B0
:20E8E000BD938612270109BD9474CCC1AFBDEEB3BDEB637C003A8603913A2E22BDEC8927E2
:20E900000B860A913A2E17BDEC192612BD947ACCC1D1BDEEB38602BDF22DBDEA50397EE8D1
:20E92000591327200713271003BDEDCDBDE688962A270139122704E9122708E57F0032BD53
:20E94000E688962A7F002A270139BDEBA3270CBDEB9D2707BDEB177F002A39BDEB17861692
:20E9600091322EDB2009BDE9B0BDE9DE7EE660BD947ACCC237BDEEB38607BDF22D20E7BDE9
:20E98000EAB57F0033BDE688962A270139BDEBA32609BDEB9D26047F002A39BDE688962A24
:20E9A000270139861691332EE47F002ABDEA0639BDEB25BDEB48BDEB2CBDEB41BDEB09BD0D
:20E9C000EB10BDEB17BDEB4FBDEB63BDEB3ABDEB1EBDEB33BDEB77BDEB7E152780397F003F
:20E9E000307F00317F00387F00397F003A7F003B7F00367F00387F002515268015273C15FD
:20EA000028F015290C39BDE9DEBDE9B0BDE921BD9474962784012717142730CCC1F3BDEEDF
:20EA2000B3BD9623122501F9BD9452122701058602972A398607972A39BDE9DEBDE9B0BDFA
:20EA4000E921152703BD947ADC46BDEEB37EE660BDE9DEBDE9B0BDE921152733BD9474CCBD
:20EA6000C17CBDEEB3BD9623122501F9BD94528601972A39BDE9DE142801BDE9B0152801DB
:20EA8000BDE921BD9623122501F9BD9452122701058602972A398607972A39BD947ACCC0C6
:20EAA0002CBDEEB37EE660CE60001C000839CE60001C000439CE60001C000239CE60001C27
:20EAC000000139CE10081C000239CE10081C000439CE10081C001039CE10081C000839CE24
:20EAE00010081C002039CE10001C008039CE10001C004039CE10001C002039CE10001C0016
:20EB00001039CE10001C000839CE60001D000839CE60001D000439CE60001D000239CE60A9
:20EB2000001D000139CE10081D000239CE10081D000439CE10081D001039CE10081D0008A9
:20EB400039CE10081D002039CE10001D008039CE10001D004012280109865B973E973D144F
:20EB6000270439CE10001D002012280109865B973E973D14270839CE10001D001039CE10AA
:20EB8000001D000839B66002841039B66002840839B66002840439B66002840239B660028D
:20EBA000840139B6100A848039B6100A84402703860039860139B6100A84202703860039F0
:20EBC000860139B6100084042703860039860139B6100084022703860039860139B61000C3
:20EBE000840139B66000840839B66000840439B61000844039B61000842039B610088402EB
:20EC000039B61008840439B61008841039B61008840839B610088420398603B7103018CEED
:20EC20000001BD9323CE10301E00800586019721397F0021F6103486C43DCE0032028FCE77
:20EC4000000A028F17970491162E038600398601398602B7103018CE0001BD9323CE103029
:20EC60001E00800586019721397F0021F6103386C43DCE0032028FCE000A028F17970491DC
:20EC8000172E038600398601398604B7103018CE0001BD9323CE10301E00800586019721E2
:20ECA000397F0021F6103186C43DCE0032028FCE000A028F17970491162E038600398601F3
:20ECC000398600B7103018CE0001BD9323CE10301E00800586019721397F0021F61031C064
:20ECE0002C86413DCE0095028FCE0001028F1780059B63912B2E038600398601398601B74C
:20ED0000103018CE0001BD9323CE10301E00800586019721397F0021F61032C02C86413D68
:20ED2000CE0095028FCE0001028F1780059B64912C2E038600398601398600B7103018CE14
:20ED40000001BD9323CE10301E00800586019721397F0021F61031C02C86413DCE009502EA
:20ED60008FCE0001028FC005DB63398601B7103018CE0001BD9323CE10301E008005860158
:20ED80009721397F0021F61032C02C86413DCE0095028FCE0001028FC005DB643997707FA3
:20EDA000006FBD95448620BD9595CE0075A60081202704BD94B0390820F3DD6FBD9544864F
:20EDC00020BD9595CE007520E4BD94B03913272079BDEBE3270413294017BD947A8681BD00
:20EDE0009496BDED3917BDED9DCCC0FCBDEEB32014BD947A8681BD9496CCC0F9BDEEB3CC26
:20EE0000C0F9BDEEB3BDEBE9270413294014868BBD9496BDED6B17BDED9DCCC0FCBDEEB33E
:20EE20002011868BBD9496CCC0F9BDEEB3CCC0F9BDEEB3132980148687BD9496CCC111BDC4
:20EE4000EEB3961EBDED9D152710398687BD9496CCC0F9BDEEB320EF13278056BD9474DCFA
:20EE600055BDEEB3DC5793300C59490C59490C59490C59490C5949CE0064028FDD59CE00BC
:20EE80003C028FD75B863C3DDD5CDC59935CD75E965BBDED9DCCC0E2BDEEB3965E81092E32
:20EEA00006CCC115BDEEB3965EBDED9DCCC0DEBDEEB33983C000D3428FBD94B0393C183C5F
:20EEC0003637200CC61086104A26FD5A26F82005BDEB8B27FB3332183838393C183C3736AB
:20EEE000BD94523233183838393C183C3736BDEB8B27FB323318383839BD947ABD947496AB
:20EF000030BDEDBA398600CEB709BD95F08600CEB70908BD95F08600CEB711BD95F086008C
:20EF2000CEB71108BD95F08600CEB713BD95F08600CEB716BD95F08600BDF22D8600BDF297
:20EF40002D8600BDF22D8600BDF22D8600BDF22D8600BDF22D8600BDF22D8600BDF22D86B2
:20EF600000BDF22D8600BDF22D8603CEB721BD95F08608CEB722BD95F0BD9452CCC0AEBDD1
:20EF8000EEB37EEF82B6B716971DFCB709DD18FCB711DD1AB6B713971C9B54813B2E569745
:20EFA0001CDC18C30001DD18961D9B10813B2E02200C803C971D961C8B01971C961D971D4A
:20EFC000961CCEB713BD95F0961DCEB716BD95F0DC1ACEB711BD95F0DC1A17CEB71108BDDF
:20EFE00095F0DC18CEB709BD95F0DC1817CEB70908BD95F039803C971CDC1AC30001DD1A8C
:20F00000209FDD46BD947ADC46BDEEB3960581092E06CCC113BDEEB39605BDED9DBD962314
:20F020001225021296058B01970581142E0220D48601970520CE960539152740BDF8A5BD91
:20F04000947ABD9474CCC0F9BDEEB3BDEB852708CCC0E6BDEEB32003BDF14ABDEB8B270851
:20F06000CCC0E6BDEEB32003BDF14ABDEB912708CCC0E6BDEEB32003BDF14ABDEB972708E4
:20F08000CCC0E6BDEEB32003BDF14ABDEB9D2708CCC0E6BDEEB32003BDF14ABDEBA32708AC
:20F0A000CCC0E6BDEEB32003BDF14ABDEBA92608CCC0E6BDEEB32003BDF14ABDEBB626086F
:20F0C000CCC0E6BDEEB32003BDF14ABDEBC32608CCC0E6BDEEB32003BDF14ABDEBD026081B
:20F0E000CCC0E6BDEEB32003BDF14ABDEBDD2708CCC0E6BDEEB32003BDF14A8681BD949698
:20F10000BDEC199604BDED9DCCC113BDEEB38687BD9496BDEC519604BDED9DCCC113BDEE34
:20F12000B3868DBD9496BDEC899604BDED9DCCC113BDEEB3BDEB8B26037EF03FBDEB8B26AF
:20F14000FBBD94527E906F7EF13CCCC115BDEEB3397EF1F19615970186099702BDF21F26F1
:20F16000F0960E970186099702BDF21F26E3960D9701865A9702BDF21F2676960C97018686
:20F18000469702BDF21F266996109701863C9702BDF21F265C960F9701863C9702BDF21FE4
:20F1A000264F96169701865A9702BDF21F264296179701865A9702BDF21F263596119701C1
:20F1C000865A9702BDF21F26289614970186019702BDF21F261B9663970186149702BDF2B6
:20F1E0001F260E9664970186149702BDF21F260139BDF85D860A97639764BDF7759663CE42
:20F20000B714BD95F09664CEB715BD95F086039715CEB706BD95F08662BDF22D7EE66096EB
:20F2200001910222022003860139860039CEB7E0E600BD95F00817E600BD95F00817E6009B
:20F24000BD95F00817E600BD95F00817E600BD95F00817E600BD95F00817E600BD95F00848
:20F2600017E600BD95F00817E600BD95F00817E600BD95F039CC003E1A93302E11BDB000F5
:20F28000BD9474CCC1C0BDEEB3CC0000DD307EE69CCC003E1A93302EF5BDB00015298014DC
:20F2A0002730BD9474CCC215BDEEB3BD9474CCC111BDEEB3961E961EBDED9DCCC113BDEE76
:20F2C000B3BDE6149654BDED9DCCC0FFBDEEB3CCC113BDEEB3962D81002708CCC15FBDEEA2
:20F2E000B32000CC0000DD307EF28EBD9474CCC27BBDEEB3BDF8A51527027F000BBD947A4B
:20F30000BDF59FBD962312250208BDF5AEBDF70620D9BDF706BD9474CCC27BBDEEB3BD949B
:20F320007ACCC28CBDEEB3BD962312250116BD947ACCC29DBDEEB3BD962312250106BDF85A
:20F340005D7EF4987C000BBD947ACCC215BDEEB3BD947ACCC29DDD44BDF4B4BD96231225CA
:20F360000205BDF5AE20E08601971EBD947ACCC111BDEEB3961EBDED9D8603D61E3DC300AB
:20F380007BC30000DD078FA60081FF26048600A70081002708CCC103BDEEB32006CCC10AE4
:20F3A000BDEEB3CCC15FBDEEB3BD962312250210DE076C008602A10026026F00DF0720AB24
:20F3C000BD947ACCC111BDEEB3961EBDED9DCCC2BFBDEEB38603D61E3DC3007BC30001DD27
:20F3E000078FA60081FF26048601A700BDED9DCCC0FFBDEEB3BD962312250210DE076C00B9
:20F400008609A1002ABA8601A70020B47C001E960E8B01911E27037EF36B7C000BBD94522D
:20F42000BD9474CCC27BBDEEB3BD947ACCC2D0BDEEB3BD96231225015FBD947ACCC215BDE1
:20F44000EEB3BD947ACCC2BFDD44BDF4B4BD962312250205BDF5AE20E97C000B8609910B9E
:20F460002AD77F000BBD947ACCC00ABDEEB3BD9474CCC27BBDEEB3BD9623122501037EE007
:20F480009EBD947ACCC369BDEEB3BD9623122502078602970B7EF442BD947ACCC37ABDEE9A
:20F4A000B3BD9623122502037EF2EBBDF775BD94527EE280BD9474CCC27BBDEEB3BD947AE9
:20F4C0008611D60B3DD344BDEEB38601910B2605960EBDED9D8602910B2617960D8101261D
:20F4E00006CCC113BDEEB3960DBDED9DCCC0FCBDEEB38603910B2617960C81012606CCC1F9
:20F5000013BDEEB3960CBDED9DCCC0FCBDEEB38604910B260B9610BDED9DCCC04EBDEEB32F
:20F520008605910B260B960FBDED9DCCC04EBDEEB38606910B26119616BDED9DCCC117BD9C
:20F54000EEB3CCC0F9BDEEB38607910B26119617BDED9DCCC117BDEEB3CCC0F9BDEEB38668
:20F5600008910B262196114981022712BDED9DCCC04EBDEEB3CCC0F9BDEEB37EF586CCC10C
:20F5800015BDEEB320E98609910B261296142708CCC103BDEEB32006CCC10ABDEEB339BDB4
:20F5A000947A8611D6153DC3C38BBDEEB3398600910B26127C0015BDF706860991152A6F63
:20F5C0007F00157EF7028601910B26107C000E8609910E2A5A8601970E7EF7028602910BC4
:20F5E00026237F0041CCFF008FD6413AA60081FF26067F00417F000D910D2E057C0041200B
:20F60000E4970D202A8603910B26277F0041CCFF158FD6413AA60081FF26067F00417F0095
:20F620000C910C2E057C004120E4970C7EF7027EF7028604910B26247F0041CCFF288FD614
:20F64000413AA600810026067F00107F004191102E057C004120E497107EF7028605910BB3
:20F6600026237F0041CCFF2F8FD6413AA600810026067F00417F000F910F2E057C00412056
:20F68000E4970F207D8606910B261396168B0A9716866391162A6B860A97167EF70286078E
:20F6A000910B261396178B0A9717866391172A52860A97177EF7028608910B26237F004190
:20F6C000CCFF4B8FD6413AA60081FF26067F00417F001191112E057C004120E49711202212
:20F6E0008609910B260F961427057F0014201386019714200DCCC02CBDEEB318CE03E8BD0B
:20F700009323BDF89B39961581002607CCC460DD42206181012607CCC8C0DD4220568102A6
:20F720002607CCCD20DD42204B81032607CCC000DD42204081042607CCD180DD42203581D9
:20F74000052607CCD5E0DD42202A81062607CCDA80DD42201F81072607CC8000DD42201401
:20F7600081082607CC8460DD42200981092605CC88C0DD4239960CCEB700BD95F0960DCEE0
:20F78000B701BD95F0960ECEB702BD95F0960FCEB703BD95F09610CEB705BD95F09615CEA8
:20F7A000B706BD95F09616CEB707BD95F09617CEB717BD95F09611CEB719BD95F09614CE46
:20F7C000B720BD95F09618CEB709BD95F0961ACEB711BD95F0BDF89BC600CEB60018CE008A
:20F7E0007B18A600BD95F00818085CD12026F239B6B700970CB6B701970DB6B702970EB6DC
:20F80000B703970FB6B7059710B6B7069715B6B7079716B6B7179717B6B7199711B6B72042
:20F820009714FCB709DD18FCB711DD1AB6B713971CB6B7149763B6B7159764B6B716971D4F
:20F84000BDF154BDF89BC600CEB60018CE007BA60018A7000818085CD12026F339863C9726
:20F860000C8655970D8603970E8614970F861E971086289716860A9717860197118600975F
:20F8800014BDF89BC600CEFF3B18CE007BA60018A7000818085CD12026F3398603D60E3DFF
:20F8A000CB03D7203918CE012CBD93237F002918CE1024181C0040BDE9DE1528FF15278012
:0DF8C000142940860097530E18CE00C83959
:209000008682BD9496BDED394F1BBDED9DCCC0FCBDEEB3CCC113BDEEB3868ABD9496BDED48
:209020006B4F1BBDED9DCCC0FCBDEEB3CCC113BDEEB3BD947486C2BD9496BDEC199604BD23
:20904000ED9DCCC113BDEEB386C7BD9496BDEC519604BDED9DCCC113BDEEB386CCBD949642
:20906000BDEC899604BDED9DCCC113BDEEB339BD9000BD9182BDEAA718CE0190BD9323BD94
:20908000EB09BD9000BD9182BDEAAE18CE0190BD9323BDEB10BD9000BD9182BDEAB518CE69
:2090A0000190BD9323BDEB17BD9000BD9182BDEABC18CE0190BD9323BDEB1EBD9000BD9122
:2090C00082BDEAC318CE0190BD9323BDEB25BD9000BD9182BDEACA18CE0190BD9323BDEBCD
:2090E0002CBD9000BD9182BDEAD118CE0190BD9323BDEB33BD9000BD9182BDEAD818CE0167
:2091000090BD9323BDEB3ABD9000BD9182BDEADF18CE0190BD9323BDEB41BD9000BD9182D7
:20912000BDEAE618CE0190BD9323BDEB48BD9000BD9182BDEAED18CE0190BD9323BDEB4F36
:20914000BD9000BD9182BDEAF418CE0190BD9323BDEB63BD9000BD9182BDEAFB18CE01902C
:20916000BD9323BDEB77BD9000BD9182BDEB0218CE0190BD9323BDEB7EBD9000BD91827EEB
:20918000906FBDEB852606BDEB097E9190BDEAA7BDEB8B2606BDEB107E919EBDEAAEBDEB18
:2091A000912606BDEB177E91ACBDEAB5BDEB972606BDEB1E7E91BABDEABCBDEB9D2606BD91
:2091C000EB257E91C8BDEAC3BDEBA32606BDEB2C7E91D6BDEACABDEBA92606BDEAD17E9199
:2091E000E4BDEB33BDEBB62606BDEAD87E91F2BDEB3ABDEBC32606BDEADF7E9200BDEB41AE
:20920000BDEBD02606BDEAE67E920EBDEB48BDEBDD2604BDEB4F39BDEAED39BDE97FBDEB96
:20922000A327F8BD945286009709BDEAA7BD92D4BDEB09BD92CCBDEAAEBD92D4BDEB10BD79
:2092400092CC7C0009BDEABCBD92D4BDEB1EBD92CCBDEAC3BD92D4BDEB25BD92CCBDEACADE
:20926000BD92D4BDEB2CBD92CCBDEAD1BD92D4BDEB33BD92CCBDEAD8BD92D4BDEB3ABD9278
:20928000CCBDEADFBD92D4BDEB41BD92CCBDEAE6BD92D4BDEB48BD92CCBDEAEDBD92D4BD26
:2092A000EB4FBD92CCBDEAF4BD92D4BDEB63BD92CCBDEAFBBD92D4BDEB77BD92CCBDEB02CC
:2092C000BD92D4BDEB7EBD92CC7E922618CE03E8BD932339BD9474CCC078BDEEB37C0009CB
:2092E0009609BDED9DCCC0F9BDEEB3BD92F2BD92CC39BDEB852703142901BDEB8B2703140A
:209300002901BDEB912703142901BDEB972703142901BDEB9D2703142901BDEBDD2703146B
:20932000290139183C3CCE01470926FD38180926F4183839183C3CCE01470926FD381809D1
:2093400026F4183839183C3CCE00200926FD38180926F418383936B66000840F9706328492
:20936000F09A06B760003918CE6002181D0040BD935618CE6002181C0080181D0080181CC5
:209380000040BD94C03918CE6002BD94C0BD94C018CE6002181D00A0181C00408630BD9342
:2093A000678630BD93678630BD93678620BD93678628BD9424BD94C08606BD9424BD94C0C9
:2093C0008614BD9424BD94C0860CBD9424BD94C08601BD9424BD94C018CE6002181C0020AC
:2093E00018CE6002181D0020181D00408640BD9424BD94C018CE6002181C0020CE9504DF2D
:209400004686409704DE46A60008DF46BD9424BD94C096044A9704810026EA18CE600218B8
:209420001C00203918CE6002970A84F0BD9356BD9441960A840F48484848BD9356BD944197
:2094400039181D0040181C0080181D0080181C00403918CE6002181D00208601BD9424BDF2
:2094600094C0BD94C018CE6002181C0020398680BD94963986C0BD94963918CE6002181DA9
:2094800000208602BD9424BD94C0BD94C018CE6002181C00203918CE6002181D0020BD94CA
:2094A00024BD94C0BD94C018CE6002181C002039A600270BBD94240886194A26FD20F139E6
:2094C00018CE0014BD93233936375F8164251A5C8064816424F9CB303617BD9424325F81E5
:2094E0000026068630BD94244F810A250F5C800A810A24F9CB303617BD9424328B30BD947E
:209500002433323904000E111F1111000A001F111F1111000A000E1111110E0003041F101B
:209520001E101F0002051F101E101F0003041F111F1111001100111111111F000E11101030
:2095400010150E037F006C7F006D7F006E86109772CE006E86039771A6009773840F8005DD
:209560002B0696738B039773967384F080502B0696738B3097739673A700097A007126D82B
:2095800078007079006F79006E79006D79006C7A007226BD39CE0075A700088C007926F82C
:2095A000CE0000966C840F27058B30977508966D444444442606D675C12027058B309776EE
:2095C00008966D840F2606D676C12027058B30977708966E444444442606D677C1202704FE
:2095E0008B309778966E840F8B3097797F007A3937183CC616F7103BE700C617F7103B1846
:20960000CE000ABD93237F103BC602F7103BA700C603F7103B18CE000ABD93237F103B1834
:2096200038333936373C183C152503BDEB8526FBBDEB8B26F618CE0019BD9323BDEB8526EA
:20964000EABDEB8B26E513274003BDE688BD968CBDEB8527037E9671BDEB8B27E918CE0056
:2096600019BD9323BDEB8B27DD142502142902201218CE0019BD9323BDEB8527C9142501B2
:189680001429021429011838383332391327200713271003BDEDCD39D1
:20A00000BDA101BD945286009709BD947ACCC03DBDEEB39609BDED9DBD9474CCC27BBDEEC7
:20A02000B3BD9623122501037EA03E7C00099609810A27037EA00A860097097EA00ACC0045
:20A0400000DD07BD947ACCC03DBDEEB39609BDED9DDC07BDEDBABD9474CCC27BBDEEB3BD14
:20A060009623122501037EA081DC07C30001DD071A83000A27037EA043CC0000DD077EA0C2
:20A08000439609B1B72126179608B1B72226102007860C972A7EE5D2860B972A7EE5D2BDC7
:20A0A000945296098107260ADC071A83000226022007860A972A7EE5D286009709BD947A1B
:20A0C000CCC03DBDEEB39609BDED9DBD9474CCC27BBDEEB3BD9623122501037EA0F17C000B
:20A0E000099609810A27037EA0BD860097097EA0BD9609810926BBBD9452860D972A7EE5C3
:20A10000D2BDEB8B26FBBD947ACCC0E8BDEEB3BD9474CCC27BBDEEB3CC0000DD30142680BD
:20A12000DC301A83000A2E05BDEB8527037EA0B2BDEB8B27EB7EA003152740BD9452CCC100
:20A140001BBDEEB3B6B721BDED9DB6B722BDED9DBD9474CCC27BBDEEB3BD962312250103FE
:20A160007EA1667EA1F4BD945286009709BD947ACCC03DBDEEB39609BDED9DBD9474CCC253
:20A180007BBDEEB3BD9623122501037EA1A17C00099609810A27037EA16D860097097EA1CB
:20A1A0006DCC0000DD07BD947ACCC03DBDEEB39609BDED9DDC07BDEDBABD9474CCC27BBDD8
:20A1C000EEB3BD9623122501037EA1E4DC07C30001DD071A83000A27037EA1A6CC0000DD60
:20A1E000077EA1A69609CEB721BD95F09608CEB722BD95F0BD9452CCC12CBDEEB37EA1FDAF
:008000017F
